:100000000C945A000C9477000C9477000C947700B1
:100010000C9477000C9477000C9477000C94770084
:100020000C9477000C9477000C9477000C94770074
:100030000C9477000C9477000C9477000C94770064
:100040000C9498000C9477000C9477000C94770033
:100050000C9477000C9477000C9477000C94770044
:100060000C9477000C947700000024272A000025C8
:10007000282B000023262904040404040404040299
:100080000202020202030303030303010204081035
:100090002040800102040810200102040810200002
:1000A0000000070002010000030406000000000039
:1000B0000000000011241FBECFEFD8E0DEBFCDBF8F
:1000C00011E0A0E0B1E0E8E5F4E002C005900D9297
:1000D000A030B107D9F711E0A0E0B1E001C01D9256
:1000E000A830B107E1F70E9479000C942A020C9421
:1000F0000000DF93CF93CDB7DEB70E943B018DE0C8
:1001000061E00E9475018DE061E00E94930168EE5C
:1001100073E080E090E00E9403018DE060E00E94C7
:10012000930168EE73E080E090E00E940301EBCF62
:100130001F920F920FB60F9211242F938F939F93BC
:10014000AF93BF938091000190910101A0910201B2
:10015000B09103018050904CAF4FBF4F809300018E
:1001600090930101A0930201B093030127C08091F5
:10017000000190910101A0910201B091030180580A
:100180009E43A040B0408093000190930101A09352
:100190000201B09303018091040190910501A091A7
:1001A0000601B09107010196A11DB11D80930401C4
:1001B00090930501A0930601B0930701809100017F
:1001C00090910101A0910201B091030181589E43D9
:1001D000A040B04060F6BF91AF919F918F912F9159
:1001E0000F900FBE0F901F9018958FB7F894209125
:1001F00004013091050140910601509107018FBF24
:10020000B901CA010895EF92FF920F931F937B01EA
:100210008C018FB7F89440910401509105016091D1
:100220000601709107018FBF2FB7F89480910401E8
:1002300090910501A0910601B09107012FBF841B89
:10024000950BA60BB70B8E159F05A007B10760F3A2
:100250001F910F91FF90EF900895019759F0FC01C5
:10026000EE0FFF1FEE0FFF1F32978FB7F8943197F5
:10027000F1F78FBF0895789484B5826084BD84B50A
:10028000816084BD85B5826085BD85B5816085BD91
:10029000EEE6F0E0808181608083E1E8F0E080813B
:1002A00082608083808181608083E0E8F0E08081EB
:1002B00081608083E1EBF0E0808184608083E0EB0B
:1002C000F0E0808181608083EAE7F0E080818460F3
:1002D000808380818260808380818160808380814F
:1002E000806880831092C1000895282F30E0C901F2
:1002F00085579F4FFC01949129583F4FF9018491F4
:10030000882381F0E82FF0E0E859FF4FE491F0E016
:10031000662329F4808190958923808308958081C4
:10032000892B80830895482F50E0CA0181569F4F42
:10033000FC012491CA0185579F4FFC0194914958B3
:100340005F4FFA0134913323C1F1222331F123307D
:1003500021F4809180008F7705C0243031F48091A2
:1003600080008F7D8093800018C0213019F484B5FF
:100370008F7704C0223021F484B58F7D84BD0DC0F9
:10038000263021F48091B0008F7705C0273029F402
:100390008091B0008F7D8093B000E32FF0E0E359AF
:1003A000FF4FE491F0E0662329F480819095892342
:1003B000808308958081892B80830895482F50E0A1
:1003C000CA0181569F4FFC012491CA0185579F4F56
:1003D000FC01949149585F4FFA013491332319F489
:1003E00020E030E035C0222331F1233021F4809128
:1003F00080008F7705C0243031F4809180008F7D9C
:100400008093800018C0213019F484B58F7704C020
:10041000223021F484B58F7D84BD0DC0263021F4B7
:100420008091B0008F7705C0273029F48091B0000B
:100430008F7D8093B000E32FF0E0EE58FF4FE49102
:10044000F0E0808120E030E0892311F021E030E00D
:08045000C9010895F894FFCFE3
:00000001FF
